
acledit.nostrip.dll:     file format pei-i386

Disassembly of section .text:

71b71000 <_DllMain@12>:
DllMain(
	HINSTANCE hinstDLL,
	DWORD     dwReason,
	LPVOID    lpvReserved)
{
71b71000:	55                   	push   %ebp
71b71001:	89 e5                	mov    %esp,%ebp
  switch (dwReason)
71b71003:	83 7d 0c 01          	cmpl   $0x1,0xc(%ebp)
71b71007:	74 09                	je     71b71012 <_DllMain@12+0x12>
  {
    case DLL_PROCESS_ATTACH:
      hDllInstance = hinstDLL;
      break;
    case DLL_THREAD_ATTACH:
      break;
    case DLL_THREAD_DETACH:
      break;
    case DLL_PROCESS_DETACH:
      break;
  }
  return TRUE;
}
71b71009:	b8 01 00 00 00       	mov    $0x1,%eax
71b7100e:	5d                   	pop    %ebp
71b7100f:	c2 0c 00             	ret    $0xc
71b71012:	8b 45 08             	mov    0x8(%ebp),%eax
71b71015:	5d                   	pop    %ebp
71b71016:	a3 00 30 b7 71       	mov    %eax,0x71b73000
71b7101b:	b8 01 00 00 00       	mov    $0x1,%eax
71b71020:	c2 0c 00             	ret    $0xc
71b71023:	90                   	nop    
71b71024:	90                   	nop    
71b71025:	90                   	nop    
71b71026:	90                   	nop    
71b71027:	90                   	nop    
71b71028:	90                   	nop    
71b71029:	90                   	nop    
71b7102a:	90                   	nop    
71b7102b:	90                   	nop    
71b7102c:	90                   	nop    
71b7102d:	90                   	nop    
71b7102e:	90                   	nop    
71b7102f:	90                   	nop    

71b71030 <_EditAuditInfo@4>:

DWORD
WINAPI
EditAuditInfo(DWORD Unknown)
{
71b71030:	55                   	push   %ebp
71b71031:	89 e5                	mov    %esp,%ebp
71b71033:	50                   	push   %eax
71b71034:	50                   	push   %eax
  UNIMPLEMENTED;
71b71035:	6a 1c                	push   $0x1c
71b71037:	68 0e 20 b7 71       	push   $0x71b7200e
71b7103c:	68 00 20 b7 71       	push   $0x71b72000
71b71041:	68 18 20 b7 71       	push   $0x71b72018
71b71046:	e8 35 01 00 00       	call   71b71180 <_DbgPrint>
  return 0;
}
71b7104b:	31 c0                	xor    %eax,%eax
71b7104d:	c9                   	leave  
71b7104e:	c2 04 00             	ret    $0x4
71b71051:	eb 0d                	jmp    71b71060 <_EditOwnerInfo@4>
71b71053:	90                   	nop    
71b71054:	90                   	nop    
71b71055:	90                   	nop    
71b71056:	90                   	nop    
71b71057:	90                   	nop    
71b71058:	90                   	nop    
71b71059:	90                   	nop    
71b7105a:	90                   	nop    
71b7105b:	90                   	nop    
71b7105c:	90                   	nop    
71b7105d:	90                   	nop    
71b7105e:	90                   	nop    
71b7105f:	90                   	nop    

71b71060 <_EditOwnerInfo@4>:

DWORD
WINAPI
EditOwnerInfo(DWORD Unknown)
{
71b71060:	55                   	push   %ebp
71b71061:	89 e5                	mov    %esp,%ebp
71b71063:	52                   	push   %edx
71b71064:	52                   	push   %edx
  UNIMPLEMENTED;
71b71065:	6a 24                	push   $0x24
71b71067:	68 0e 20 b7 71       	push   $0x71b7200e
71b7106c:	68 41 20 b7 71       	push   $0x71b72041
71b71071:	68 18 20 b7 71       	push   $0x71b72018
71b71076:	e8 05 01 00 00       	call   71b71180 <_DbgPrint>
  return 0;
}
71b7107b:	31 c0                	xor    %eax,%eax
71b7107d:	c9                   	leave  
71b7107e:	c2 04 00             	ret    $0x4
71b71081:	eb 0d                	jmp    71b71090 <_EditPermissionInfo@4>
71b71083:	90                   	nop    
71b71084:	90                   	nop    
71b71085:	90                   	nop    
71b71086:	90                   	nop    
71b71087:	90                   	nop    
71b71088:	90                   	nop    
71b71089:	90                   	nop    
71b7108a:	90                   	nop    
71b7108b:	90                   	nop    
71b7108c:	90                   	nop    
71b7108d:	90                   	nop    
71b7108e:	90                   	nop    
71b7108f:	90                   	nop    

71b71090 <_EditPermissionInfo@4>:

DWORD
WINAPI
EditPermissionInfo(DWORD Unknown)
{
71b71090:	55                   	push   %ebp
71b71091:	89 e5                	mov    %esp,%ebp
71b71093:	51                   	push   %ecx
71b71094:	51                   	push   %ecx
  UNIMPLEMENTED;
71b71095:	6a 2c                	push   $0x2c
71b71097:	68 0e 20 b7 71       	push   $0x71b7200e
71b7109c:	68 4f 20 b7 71       	push   $0x71b7204f
71b710a1:	68 18 20 b7 71       	push   $0x71b72018
71b710a6:	e8 d5 00 00 00       	call   71b71180 <_DbgPrint>
  return 0;
}
71b710ab:	31 c0                	xor    %eax,%eax
71b710ad:	c9                   	leave  
71b710ae:	c2 04 00             	ret    $0x4
71b710b1:	eb 0d                	jmp    71b710c0 <_FMExtensionProcW@12>
71b710b3:	90                   	nop    
71b710b4:	90                   	nop    
71b710b5:	90                   	nop    
71b710b6:	90                   	nop    
71b710b7:	90                   	nop    
71b710b8:	90                   	nop    
71b710b9:	90                   	nop    
71b710ba:	90                   	nop    
71b710bb:	90                   	nop    
71b710bc:	90                   	nop    
71b710bd:	90                   	nop    
71b710be:	90                   	nop    
71b710bf:	90                   	nop    

71b710c0 <_FMExtensionProcW@12>:

LONG
WINAPI
FMExtensionProcW(HWND hWnd,
                 WORD wEvent,
		 LONG lParam)
{
71b710c0:	55                   	push   %ebp
71b710c1:	89 e5                	mov    %esp,%ebp
71b710c3:	50                   	push   %eax
71b710c4:	50                   	push   %eax
  UNIMPLEMENTED;
71b710c5:	6a 36                	push   $0x36
71b710c7:	68 0e 20 b7 71       	push   $0x71b7200e
71b710cc:	68 62 20 b7 71       	push   $0x71b72062
71b710d1:	68 18 20 b7 71       	push   $0x71b72018
71b710d6:	e8 a5 00 00 00       	call   71b71180 <_DbgPrint>
  return 0;
}
71b710db:	31 c0                	xor    %eax,%eax
71b710dd:	c9                   	leave  
71b710de:	c2 0c 00             	ret    $0xc
71b710e1:	eb 0d                	jmp    71b710f0 <_SedDiscretionaryAclEditor@52>
71b710e3:	90                   	nop    
71b710e4:	90                   	nop    
71b710e5:	90                   	nop    
71b710e6:	90                   	nop    
71b710e7:	90                   	nop    
71b710e8:	90                   	nop    
71b710e9:	90                   	nop    
71b710ea:	90                   	nop    
71b710eb:	90                   	nop    
71b710ec:	90                   	nop    
71b710ed:	90                   	nop    
71b710ee:	90                   	nop    
71b710ef:	90                   	nop    

71b710f0 <_SedDiscretionaryAclEditor@52>:

DWORD
WINAPI
SedDiscretionaryAclEditor(HWND hWndOwner,
                          HINSTANCE hInstance,
                          LPCWSTR lpMachineName,
                          PACL_DLG_CONTROL pAclDlgControl,
                          PACL_EDIT_CONTROL pAclEditControl,
                          LPCWSTR lpObjectName,
                          PACL_CHANGE pChangeCallback,
                          PVOID pChangeCallbackContext,
                          PSECURITY_DESCRIPTOR pObjectSecurity,
                          BOOL bNoReadPermission,
                          BOOL bReadOnly,
                          LPDWORD lpdwChangeContextStatus,
                          DWORD Reserved)
{
71b710f0:	55                   	push   %ebp
71b710f1:	89 e5                	mov    %esp,%ebp
71b710f3:	50                   	push   %eax
71b710f4:	50                   	push   %eax
  UNIMPLEMENTED;
71b710f5:	6a 4a                	push   $0x4a
71b710f7:	68 0e 20 b7 71       	push   $0x71b7200e
71b710fc:	68 73 20 b7 71       	push   $0x71b72073
71b71101:	68 18 20 b7 71       	push   $0x71b72018
71b71106:	e8 75 00 00 00       	call   71b71180 <_DbgPrint>
  return 0;
}
71b7110b:	31 c0                	xor    %eax,%eax
71b7110d:	c9                   	leave  
71b7110e:	c2 34 00             	ret    $0x34
71b71111:	eb 0d                	jmp    71b71120 <_SedTakeOwnership@56>
71b71113:	90                   	nop    
71b71114:	90                   	nop    
71b71115:	90                   	nop    
71b71116:	90                   	nop    
71b71117:	90                   	nop    
71b71118:	90                   	nop    
71b71119:	90                   	nop    
71b7111a:	90                   	nop    
71b7111b:	90                   	nop    
71b7111c:	90                   	nop    
71b7111d:	90                   	nop    
71b7111e:	90                   	nop    
71b7111f:	90                   	nop    

71b71120 <_SedTakeOwnership@56>:

DWORD
WINAPI
SedTakeOwnership(HWND hWndOwner,
                 HINSTANCE hInstance,
                 LPCWSTR lpMachineName,
                 LPCWSTR lpObjectType,
                 LPCWSTR lpObjectName,
                 DWORD dwObjectCount,
                 PACL_CHANGE pChangeCallback,
                 PVOID pChangeCallbackContext,
                 PSECURITY_DESCRIPTOR pObjectSecurity,
                 BOOL NoReadPermission,
                 BOOL NoOwnerChange,
                 LPDWORD lpdwChangeContextStatus,
                 PACL_HELP_CONTROL pHelpInfo,
                 DWORD Reserved)
{
71b71120:	55                   	push   %ebp
71b71121:	89 e5                	mov    %esp,%ebp
71b71123:	50                   	push   %eax
71b71124:	50                   	push   %eax
  UNIMPLEMENTED;
71b71125:	6a 5f                	push   $0x5f
71b71127:	68 0e 20 b7 71       	push   $0x71b7200e
71b7112c:	68 8d 20 b7 71       	push   $0x71b7208d
71b71131:	68 18 20 b7 71       	push   $0x71b72018
71b71136:	e8 45 00 00 00       	call   71b71180 <_DbgPrint>
  return 0;
}
71b7113b:	31 c0                	xor    %eax,%eax
71b7113d:	c9                   	leave  
71b7113e:	c2 38 00             	ret    $0x38
71b71141:	eb 0d                	jmp    71b71150 <_SedSystemAclEditor@48>
71b71143:	90                   	nop    
71b71144:	90                   	nop    
71b71145:	90                   	nop    
71b71146:	90                   	nop    
71b71147:	90                   	nop    
71b71148:	90                   	nop    
71b71149:	90                   	nop    
71b7114a:	90                   	nop    
71b7114b:	90                   	nop    
71b7114c:	90                   	nop    
71b7114d:	90                   	nop    
71b7114e:	90                   	nop    
71b7114f:	90                   	nop    

71b71150 <_SedSystemAclEditor@48>:

DWORD
WINAPI
SedSystemAclEditor(HWND hWndOwner,
                   HINSTANCE hInstance,
                   LPCWSTR lpMachineName,
                   PACL_DLG_CONTROL pAclDlgControl,
                   PACL_EDIT_CONTROL pAclEditControl,
                   LPCWSTR lpObjectName,
                   PACL_CHANGE pChangeCallback,
                   PVOID pChangeCallbackContext,
                   PSECURITY_DESCRIPTOR pObjectSecurity,
                   BOOL bNoReadPermission,
                   LPDWORD lpdwChangeContextStatus,
                   DWORD Reserved)
{
71b71150:	55                   	push   %ebp
71b71151:	89 e5                	mov    %esp,%ebp
71b71153:	50                   	push   %eax
71b71154:	50                   	push   %eax
  UNIMPLEMENTED;
71b71155:	6a 72                	push   $0x72
71b71157:	68 0e 20 b7 71       	push   $0x71b7200e
71b7115c:	68 9e 20 b7 71       	push   $0x71b7209e
71b71161:	68 18 20 b7 71       	push   $0x71b72018
71b71166:	e8 15 00 00 00       	call   71b71180 <_DbgPrint>
  return 0;
}
71b7116b:	31 c0                	xor    %eax,%eax
71b7116d:	c9                   	leave  
71b7116e:	c2 30 00             	ret    $0x30
71b71171:	90                   	nop    
71b71172:	90                   	nop    
71b71173:	90                   	nop    
71b71174:	90                   	nop    
71b71175:	90                   	nop    
71b71176:	90                   	nop    
71b71177:	90                   	nop    
71b71178:	90                   	nop    
71b71179:	90                   	nop    
71b7117a:	90                   	nop    
71b7117b:	90                   	nop    
71b7117c:	90                   	nop    
71b7117d:	90                   	nop    
71b7117e:	90                   	nop    
71b7117f:	90                   	nop    

71b71180 <_DbgPrint>:
71b71180:	ff 25 38 50 b7 71    	jmp    *0x71b75038
71b71186:	90                   	nop    
71b71187:	90                   	nop    
	...

71b71190 <__CTOR_LIST__>:
71b71190:	ff                   	(bad)  
71b71191:	ff                   	(bad)  
71b71192:	ff                   	(bad)  
71b71193:	ff 00                	incl   (%eax)
71b71195:	00 00                	add    %al,(%eax)
	...

71b71198 <__DTOR_LIST__>:
71b71198:	ff                   	(bad)  
71b71199:	ff                   	(bad)  
71b7119a:	ff                   	(bad)  
71b7119b:	ff 00                	incl   (%eax)
71b7119d:	00 00                	add    %al,(%eax)
	...
